:100000000AC01895189515C1189525C21895189508
:100010001895189518958FED8DBFC0ECE0EC4E2E1D
:10002000DD275D2EEEE7F0E0A0E6B0E088278D93B7
:100030003197E9F766248FEF87BB8FE381BB80E0C0
:1000400080937E0080E08FBD81E08EBD89B788609F
:1000500089BF89B7806889BF78948FE788BB83E4BC
:1000600082BB84E090E0B3D285E482BB84E090E080
:10007000AED289E482BB84E090E0A9D281E582BB64
:1000800084E090E0A4D2A0E80D911C91013050E0F2
:10009000150709F0E2CFAEE78C918F5F8C9300914A
:1000A0007E000C3009F018C080E080937E0080E074
:1000B00090E0A4E78D939C93A0E7E4E7F0E0B9D249
:1000C00080E08093700080E08093710080E08093F6
:1000D000720080E38093730081E080937F00009141
:1000E0007F00043010F009F010C0AFE7AD90AFE62C
:1000F000AA0D8C91AFE7AD90A1E8AA0D8C93AFE764
:100100008C918F5F8C9309F0EACF81E080937F0020
:1001100000917F000F3F10F009F08AC081E08093CA
:100120008A0000918A00043010F009F07BC0AAE830
:10013000AD90A1E8AA0D8C91A6E88D9388278C93A9
:10014000A6E80D911C91003350E0150709F003C09B
:100150008FE388BB4AC0013350E0150709F003C0A4
:1001600086E088BB42C0023350E0150709F003C0A7
:100170008BE588BB3AC0033350E0150709F003C094
:100180008FE488BB32C0043350E0150709F003C088
:1001900086E688BB2AC0053350E0150709F003C086
:1001A0008DE688BB22C0063350E0150709F003C076
:1001B0008DE788BB1AC0073350E0150709F003C06C
:1001C00087E288BB12C0083350E0150709F003C06E
:1001D0008FE788BB0AC0093350E0150709F003C058
:1001E0008FE688BB02C080E088BBAAE88C91A2E3BE
:1001F00007D2FCD19C91982B9C93EF93FF93ECE852
:10020000F1E0DCD1FF91EF91AAE88C91A2E3F8D163
:10021000EDD18C9189238C93AAE88C918F5F8C937C
:1002200009F07FCFAFE78C918F5F8C9309F070CF8F
:1002300032CF0F921F922F923F924F925F927F92F6
:10024000AF92BF920F931F932F933F934F935F9360
:100250006F937F938F939F93AF93BF93CF93DF93CE
:10026000EF93FF938FB78F93F89481E090E0A0E82D
:100270008D939C9380E080937E00ACE48D919C9163
:10028000A0E68D939C9380E090E090934D00809346
:100290004C00A2E68D919C91A4E68D939D938827B6
:1002A0008D938C9380E090E0A2E68D939C93A4E6DE
:1002B0000D911D912D913C9140E050E061E070E086
:1002C00009D1A8E60D931D932D933D93A8E60D91BA
:1002D0001D912D913C91A0E64D915C916627772769
:1002E00095D1A8E60D931D932D933D9300E018E35F
:1002F0002CE93CE1A8E64D915D916D917C91EFD0A8
:10030000ACE64D935D936D937D93AAE78D919C919F
:10031000ACE78D939C93A8E78D919C91AAE78D9370
:100320009C93A6E78D919C91A8E78D939C93ACE656
:100330008D919C91A6E78D939C93A6E70D911C91BE
:1003400022273327A8E74D915C91662777275ED156
:10035000A0E70D931D932D933D93AAE70D911C915A
:1003600022273327ACE74D915C91662777274ED142
:10037000ACE60D931D932D933D93A0E70D911D9138
:100380002D913C91ACE64D915D916D917C913ED16A
:10039000ACE60D931D932D933D93ACE60D911D910D
:1003A0002D913C9144E050E060E070E098D0ACE6E4
:1003B0004D935D936D937D93ACE68D919C91A4E7F5
:1003C0008D939C93A4E70D911C910F3057E2150774
:1003D00010F009F001C002C0909A01C09098A0E707
:1003E000E4E7F0E026D100917300003009F016C078
:1003F00080917200809373008091710080937200ED
:10040000809170008093710080E080937000009173
:100410007300003010F009F001C0EACF78948F919A
:100420008FBFFF91EF91DF91CF91BF91AF919F91DE
:100430008F917F916F915F914F913F912F911F917C
:100440000F91BF90AF907F905F904F903F902F9013
:100450001F900F9018950F921F922F923F924F92DC
:100460005F927F92AF92BF920F931F932F933F9310
:100470004F935F936F937F938F939F93AF93BF93AC
:10048000CF93DF93EF93FF938FB78F93A2E61CD0A8
:100490008F918FBFFF91EF91DF91CF91BF91AF917E
:1004A0009F918F917F916F915F914F913F912F918C
:1004B0001F910F91BF90AF907F905F904F903F90B2
:1004C0002F901F900F901895ED91FC913196FC9311
:1004D000EE93089550D00AD000FC05D008954BD07B
:1004E00020D001F8F9CF52D05AD00895842F952FFB
:1004F000A62FB72F4427552766277727F1E2889440
:1005000009C020F4480F591F6A1F7B1F7695679515
:10051000579547953795279517950795FA9589F734
:100520000895842F952FA62FB72FE894452B462B9F
:10053000472B11F468940895402F512F622F732F89
:100540000027112722273327F0E2440F551F661F8B
:10055000771F001F111F221F331F081B190B2A0BA7
:100560003B0B416028F4080F191F2A1F3B1F4E7FC9
:10057000FA9559F708950024E89477FF02C006D051
:10058000689400F809D010F80124089512D04F5F44
:100590005F4F6F4F7F4F0895E89437FF08950095A0
:1005A0001095209530950F5F1F4F2F4F3F4F689448
:1005B0000895409550956095709508953197F1F79D
:1005C0000895689462F80895E89462F80895EF93A6
:1005D000FF93EE27E82BE92B31F0E0EDF7E03197C0
:1005E000F1F70197D1F7FF91EF91089591E08823FA
:1005F00021F08894991F8A95E9F7892F909508959D
:10060000883018F011968850FBCF0895040F151FFD
:10061000261F371F0895000F111F221F331F089533
:1006200000951095209530950F5F1F4F2F4F3F4F2E
:100630000895019110810EC0019111912191308195
:100640000BC00191108117FF05C03FEF2FEF04C0D1
:10065000008111272227332737FF03C0E1DF8DE216
:100660008D93CF93DF93CF92DF92EF92AA24BB2496
:10067000CC24DD24EE2440E2CAE0DD2755E093E3FC
:100680008881890F87FD9F7083FD907F891B8993E7
:100690005A95A9F7C0DFAA1CBB1CCC1CDD1CEE1CA4
:1006A0004A9551F7E894EFE0FF2782910ED0EB30A6
:1006B000E0F71EF068948A2D0CD088278D93EF9078
:1006C000DF90CF90DF91CF910895982F829501D040
:1006D000892F8F70805D26F0803309F40895689427
:0406E0008D93089559
:00000001FF
